:020000040000FA
:100200006DEF0DF01200000000018B918B93200E1A
:100210008C6F040E916F8DC08FF08EC090F08F1F89
:10022000901F120000018BB110D00001AEB1B5D10A
:100230000001B56B0001010EB46F00019A0EB36F9F
:10024000CEEC0AF000018B8112008BB30DD00001BF
:10025000AEB1A3D10001B26B00019A0EB16FC2EC36
:100260000AF000018B831200915102E09107120005
:10027000040E916F8C5117E00001AEA986D10001E8
:100280008C07ADC028F0296A28BE29688D51282422
:100290008D6F8E5129208E6F030E8D27000E8E23B9
:1002A0000001AE9972D1200E1F6E206A8DC01AF027
:1002B0008EC01BF0A6EC0CF01AC08DF01BC08EF0A7
:1002C0001AC028F01BC029F0200E1F6E206AA6EC71
:1002D0000CF016C028F017C029F01750000AE8AE3D
:1002E00002D0293405D0100ED8802854000E29548D
:1002F00004E200018D2B000E8E2300018D518F1919
:1003000002E18E51901901E13BD18DC08FF08EC07A
:1003100090F0200E9D6F9C6F9B6F9A6F996F990E56
:10032000E66E000EE66E8DC0E6FF8EC0E6FFB3EC13
:1003300009F0E552E552E552E5520001AB0E866F39
:100340000E0E876F000E886FA8EC03F00001050EFB
:10035000986F0001980E846F000E856F37EC03F0E4
:100360000001200E9D6F9C6F9B6F9A6F996F8DC0DF
:1003700028F08EC029F0030ED89028362936E806DA
:10038000FBE10A0E1F6E206A28C01AF029C01BF07C
:10039000A6EC0CF01AC028F01BC029F0200E28266D
:1003A000000E2922285000018D25946F29508E219E
:1003B000956F8DC028F08EC029F0030ED890283696
:1003C0002936E806FBE10A0E1F6E206A28C01AF0E3
:1003D00029C01BF0A6EC0CF016C028F017C029F0BD
:1003E0001750000AE8AE02D0293405D0050ED88097
:1003F0002854000E295404E20001942B000E95238A
:10040000990EE66E000EE66E94C0E6FF95C0E6FF1C
:10041000B3EC09F0E552E552E552E5520001B30EA6
:10042000866F0E0E876F000E886FA8EC03F0000138
:10043000050E986F0001980E846F000E856F37ECE3
:1004400003F00001200E9D6F9C6F9B6F9A6F996F58
:10045000110E8D25926F010E8E21936F990EE66E0F
:10046000000EE66E92C0E6FF93C0E6FFB3EC09F023
:10047000E552E552E552E5520001BB0E866F0E0EC5
:10048000876F000E886FA8EC03F00001050E986FCF
:100490000001980E846F000E856F37EC03F00001A9
:1004A000200E9D6F9C6F9B6F9A6F996F8DC028F087
:1004B0008EC029F0030ED89028362936E806FBE1D5
:1004C0000A0E1F6E206A28C01AF029C01BF0A6EC85
:1004D0000CF01AC028F01BC029F0EC0E2826010EE3
:1004E0002922285000018D25966F29508E21976F63
:1004F0008DC028F08EC029F0030ED89028362936FA
:10050000E806FBE10A0E1F6E206A28C01AF029C017
:100510001BF0A6EC0CF016C028F017C029F01750FD
:10052000000AE8AE02D0293405D0050ED880285440
:10053000000E295404E20001962B000E9723990E19
:10054000E66E000EE66E96C0E6FF97C0E6FFB3ECDF
:1005500009F0E552E552E552E5520001C30E866FFF
:100560000E0E876F000E886FA8EC03F00001050ED9
:10057000986F0001980E846F000E856F37EC03F0C2
:100580000001200E8C6F8D6B8E6B0001AEB105D01B
:1005900000019A0EB66FDCEC0AF0120083C082F004
:1005A000000E0001796F7A6B776F786B8193AB6A7D
:1005B000900EAB6EAC6A240EAC6E83C0AFFF010C24
:1005C000120000018151020B43E0AC50020B40E0ED
:1005D0007DC0E9FF7EC0EAFFEF50AD6E7F077F511F
:1005E00034E17951771911E17A5178190EE177C028
:1005F00007F078C008F09AEC08F0000E0001796F5F
:100600007A6B776F786B819323D077C0E9FF78C0DE
:10061000EAFFEE52EECF7BF0EDCF7CF0030E7B25B0
:100620007D6F000E7C217E6F77C0E9FF78C0EAFF06
:10063000EFCF7FF077C007F078C008F09AEC08F0B1
:100640007BC077F07CC078F003D07D2B000E7E233A
:10065000AB50040B03E1AB50020B08E0AB6A900E09
:10066000AB6EAC6A240EAC6E82C0AFFF120084C0C9
:10067000E9FF85C0EAFFEF50286E296A010E28269F
:10068000000E2922020E28240001006F37EC08F02A
:10069000F3CF7BF0F4CF7CF00001F350F41057E07F
:1006A0007751781119E17BC079F07CC07AF07BC07A
:1006B00077F07CC078F084C0E9FF85C0EAFFEFCF17
:1006C0007FF0010E77257D6F000E78217E6F020E80
:1006D0007D27000E7E231AD079C0E9FF7AC0EAFF99
:1006E000EE527BC0EEFF7CC0EDFF84C0E9FF85C009
:1006F000EAFFEF50E66E79C0E9FF7AC0EAFFE55203
:10070000E750EF6E7BC079F07CC07AF084C0E9FFDF
:1007100085C0EAFFEF500001A26FA36B030E00013A
:100720007B250001A06F000E00017C210001A16F5C
:10073000010E0001842500019E6F000E000185213D
:1007400000019F6F2CEC04F000018183010C000C70
:1007500086C0F6FF87C0F7FF88C0F8FF0800F55095
:10076000286E296A010E2826000E2922020E28244E
:100770000001006F37EC08F0F3CF7BF0F4CF7CF092
:100780000001F350F41061E0775178111CE17BC057
:1007900079F07CC07AF07BC077F07CC078F086C0BE
:1007A000F6FF87C0F7FF88C0F8FF0800F5CF7FF09D
:1007B000010E77257D6F000E78217E6F020E7D275A
:1007C000000E7E231DD079C0E9FF7AC0EAFFEE5209
:1007D0007BC0EEFF7CC0EDFF86C0F6FF87C0F7FF51
:1007E00088C0F8FF0800F550E66E79C0E9FF7AC0CE
:1007F000EAFFE552E750EF6E7BC079F07CC07AF0FB
:1008000086C0F6FF87C0F7FF88C0F8FF0800F550E4
:100810000001A96FAA6B030E00017B250001A76FE1
:10082000000E00017C210001A86F86C0A4F087C0E3
:10083000A5F088C0A6F00001A42B000EA523A623D6
:10084000FBEC04F000018183010C000C12009EAA55
:1008500002D0AE501200000C0001A251A31101E120
:10086000C9D0040EA25D000EA35911E29EC0E9FF9B
:100870009FC0EAFFEF50A0C0E9FFA1C0EAFFEF6E02
:10088000A02B000EA1239E2B9F23A207B1D0080E00
:10089000A25D000EA35922E29EC0E9FF9FC0EAFFBD
:1008A000EECF28F0EECF29F0EECF2AF0EFCF2BF0ED
:1008B000A0C0E9FFA1C0EAFF28C0EEFF29C0EEFFFB
:1008C0002AC0EEFF2BC0EEFF040EA027000EA123CE
:1008D000040E9E27000E9F23040E88D0100EA25DEA
:1008E000000EA35932E29EC0E9FF9FC0EAFFEECF9F
:1008F00028F0EECF29F0EECF2AF0EECF2BF0EECF9E
:100900002CF0EECF2DF0EECF2EF0EFCF2FF0A0C0D9
:10091000E9FFA1C0EAFF28C0EEFF29C0EEFF2AC010
:10092000EEFF2BC0EEFF2CC0EEFF2DC0EEFF2EC061
:10093000EEFF2FC0EEFF080EA027000EA123080E29
:100940009E27000E9F23080E51D09EC0E9FF9FC036
:10095000EAFFEECF28F0EECF29F0EECF2AF0EECF6F
:100960002BF0EECF2CF0EECF2DF0EECF2EF0EECF21
:100970002FF0EECF30F0EECF31F0EECF32F0EECF01
:1009800033F0EECF34F0EECF35F0EECF36F0EFCFE0
:1009900037F0A0C0E9FFA1C0EAFF28C0EEFF29C0E0
:1009A000EEFF2AC0EEFF2BC0EEFF2CC0EEFF2DC0E5
:1009B000EEFF2EC0EEFF2FC0EEFF30C0EEFF31C0C5
:1009C000EEFF32C0EEFF33C0EEFF34C0EEFF35C0A5
:1009D000EEFF36C0EEFF37C0EEFF100EA027000E70
:1009E000A123100E9E27000E9F23100EA25F000E63
:1009F000A35B32D712000001A951AA1101E188D0EE
:100A0000040EA95D000EAA5915E2A4C0F6FFA5C008
:100A1000F7FFA6C0F8FF0800F550A7C0E9FFA8C07F
:100A2000EAFFEF6EA72B000EA823A42BA523A62375
:100A3000A9076CD0080EA95D000EAA5929E2A4C02E
:100A4000F6FFA5C0F7FFA6C0F8FF0900F5CF28F014
:100A50000900F5CF29F00900F5CF2AF00800F5CFFD
:100A60002BF0A7C0E9FFA8C0EAFF28C0EEFF29C00D
:100A7000EEFF2AC0EEFF2BC0EEFF040EA727000EEC
:100A8000A823040EA427000EA523A623040E3CD001
:100A9000A4C0F6FFA5C0F7FFA6C0F8FF0900F5CF78
:100AA00028F00900F5CF29F00900F5CF2AF0090058
:100AB000F5CF2BF00900F5CF2CF00900F5CF2DF084
:100AC0000900F5CF2EF00800F5CF2FF0A7C0E9FF01
:100AD000A8C0EAFF28C0EEFF29C0EEFF2AC0EEFF43
:100AE0002BC0EEFF2CC0EEFF2DC0EEFF2EC0EEFFA0
:100AF0002FC0EEFF080EA727000EA823080EA4277C
:100B0000000EA523A623080EA95F000EAA5B73D7CB
:100B10001200010EC26EC16A830EC06E0001080E83
:100B2000606F61C063F062C064F0631F641F1200F5
:100B30009EAC49D19E9C0001605108E06007615164
:100B4000C324616F6251C420626F120061C028F03B
:100B500062C029F0030ED89029322832E804FBE164
:100B600028C061F029C062F000012850631902E139
:100B70006251641901E121D161C063F062C064F087
:100B80000001F80E866F0E0E876F000E886FA8ECBE
:100B900003F00001200E766F756F746F736F726FC4
:100BA000720EE66E000EE66E61C0E6FF62C0E6FF02
:100BB000B3EC09F0E552E552E552E5520001050EAD
:100BC000716F0001710E846F000E856F37EC03F0BA
:100BD0000001EF0E866F0E0E876F000E886FA8EC77
:100BE00003F00001200E766F756F746F726F050E43
:100BF0001A6E1B6A61C01FF062C020F0CCEC0CF0D2
:100C000018C065F019C066F01F68030E206E18C08A
:100C10001AF019C01BF046EC0DF01AC065F01BC0AD
:100C200066F00001676B686B720EE66E000EE66E92
:100C30001AC0E6FF1BC0E6FFB3EC09F0E552E5522F
:100C4000E552E55200012E0E736F050E1A6E1B6AF7
:100C500061C01FF062C020F0CCEC0CF018C065F051
:100C600019C066F01F68030E206E18C01AF019C074
:100C70001BF046EC0DF016C065F017C066F00001E1
:100C80000A0E6603F3CF66F06503F3CF65F0F45008
:100C90006627676B686BF3CF69F066C06AF067C060
:100CA0006BF068C06CF01D68030E1E6E1F6A206A30
:100CB000F3CF18F066C019F067C01AF068C01BF0D7
:100CC00022EC0DF018C069F019C06AF01AC06BF080
:100CD0001BC06CF0740EE66E000EE66E18C0E6FFE8
:100CE00019C0E6FFB3EC09F0E552E552E552E552D2
:100CF00065C069F066C06AF067C06BF068C06CF0F0
:100D00001D68030E1E6E1F6A206A65C018F066C05B
:100D100019F067C01AF068C01BF022EC0DF014C087
:100D200069F015C06AF016C06BF017C06CF00A0EBF
:100D30001D6E1E6A1F6A206A14C018F015C019F0D3
:100D400016C01AF017C01BF0EAEC0CF014C069F0E2
:100D500015C06AF016C06BF017C06CF01D68030E6A
:100D60001E6E1F6A206A14C018F015C019F016C054
:100D70001AF017C01BF022EC0DF018C069F019C072
:100D80006AF01AC06BF01BC06CF0750EE66E000EB8
:100D9000E66E18C0E6FF19C0E6FFB3EC09F0E552B5
:100DA000E552E552E5520001050E716F0001710E2A
:100DB000846F000E856F37EC03F00001080E606F42
:100DC000616B626B1200C2821200031B5B66031B25
:100DD0005B4A020D0A5B504943313846383732309E
:100DE0002044656D6F20426F6172640A0D004D6989
:100DF00063726F6368697020546563686E6F6C6FAF
:100E0000677920496E632E0A0D0044656D6F206678
:100E100069726D776172652076312E30300A0D006F
:100E200041756775737420362C20323030340A0DCA
:100E3000000B526F737320466F736C65720A0D005E
:100E4000691B5B373B316654656D70657261747503
:100E50007265202843656C73697573293A0A0D0021
:100E600054656D706572617475726520284661689D
:100E700072656E68656974293A0A0D0054656D7073
:100E80006572617475726520284B656C76696E2990
:100E90003A0A0D0054656D70657261747572652053
:100EA0002852616E6B696E65293A00071B5B373B00
:100EB000323766071B5B383B323766071B5B393BB3
:100EC000323766081B5B31303B323766211B5B31A2
:100ED000323B3166504F5420566F6C746167653AEF
:100EE000200A0D00504F542056616C75653A000879
:100EF0001B5B31323B313466081B5B31333B313491
:100F0000663F1B5B31353B31664C4544733A2020CC
:100F1000204431202020443220202044332020202F
:100F200044342020204435202020443620202044F2
:100F30003720202044380A0D005374617475733AC9
:100F40002000071B5B31363B3966054F6E202020A1
:100F500000054F6666202000131B5B31383B31666D
:100F6000427574746F6E205242303A2000081B5B49
:100F700031383B3133660B507265737365642020E2
:100F80002020000B4E6F74207072657373656400CF
:100F9000241B5B32323B31665072657373202762CB
:100FA0002720746F20656E74657220626F6F7420E5
:100FB0006D6F64652E003F1B5B373B3166456E7479
:100FC0006572696E6720626F6F74206D6F64652053
:100FD00077696C6C20666F72636520746865206445
:100FE000656D6F206669726D7761726520746F2020
:100FF00073746F700A0D005366756E6374696F6E5B
:10100000696E672E20416E792070726F6772616D14
:101010006D696E67206F7065726174696F6E2074A0
:1010200068657265206166746572206D61790A0D6C
:101030000064657374726F79207468652064656DEF
:101040006F20636F64652E0A0D0A0D001F446F2028
:10105000796F752077616E7420746F20656E74658A
:101060007220626F6F74206D6F64653F00FF0050E7
:101070007E0810E3000E016E0A0E026E01C0E9FF49
:1010800002C0EAFFEF50056EE8507F0BFF0F066EBF
:10109000055003E1F36AF46A120005BE42D006501F
:1010A000D880005408E201C00DF002C00EF074D8E0
:1010B0000009E4E136D00650005C0EE101C0E9FF12
:1010C00002C0EAFFEF8E010E0124286E000E0220FE
:1010D00028C0F3FFF46E1200810E0024E66E01C0FA
:1010E000E9FF02C0EAFFE552E750EF6E010E01246E
:1010F000036E000E0220046E0028296AE8500126C3
:10110000295002220050065CE66E01C0E9FF02C0D1
:10111000EAFFE552E750EF6E03C0F3FF04C0F4FFAF
:10112000120005507F0B286E296AE85001262950CD
:101130000222A4D707C0E9FF08C0EAFFE906000EB3
:10114000EA5AEF9E1200000E096E0A0E0A6E0B6834
:10115000020E0C6E7F0ED8800B54000E0C540EE263
:1011600009C0E9FF0AC0EAFF7F0EEF6E0926000EF4
:101170000A227F0E0B5E000E0C5AECD709C0E9FF65
:101180000AC0EAFF0BC0EFFF09500B24E96E0A50BA
:101190000C20EA6EEF6A12000DC0E9FF0EC0EAFFF4
:1011A000EF5000010D240F6F000E0E20106FEF5056
:1011B000116E0FC0E9FF10C0EAFFEF50126EE85049
:1011C00001E1000C1150800B03E11250800B01E093
:1011D000000C11507F0B7F0801E1000C115012240C
:1011E000136EE8507F081BE20DC0E9FF0EC0EAFF56
:1011F0007F0EEF6E0D26000E0E221250296A12503D
:101200000F26295010220D500F5C286E0E501058DA
:101210000DC0E9FF0EC0EAFF28C0EFFF7F0C0DC034
:10122000E9FF0EC0EAFF13C0EFFFEF5012008C6819
:10123000956A12000001420E866F0F0E876F000E36
:10124000886FA8EC03F08CA007D000014A0E866FCF
:101250000F0E876F000E06D00001510E866F0F0E25
:10126000876F000E886FA8EC03F08CA207D00001F6
:101270004A0E866F0F0E876F000E06D00001510ECA
:10128000866F0F0E876F000E886FA8EC03F08CA49A
:1012900007D000014A0E866F0F0E876F000E06D032
:1012A0000001510E866F0F0E876F000E886FA8EC3D
:1012B00003F08CA607D000014A0E866F0F0E876FD1
:1012C000000E06D00001510E866F0F0E876F000EC4
:1012D000886FA8EC03F08CA807D000014A0E866F37
:1012E0000F0E876F000E06D00001510E866F0F0E95
:1012F000876F000E886FA8EC03F08CAA07D000015E
:101300004A0E866F0F0E876F000E06D00001510E39
:10131000866F0F0E876F000E886FA8EC03F08CAC01
:1013200007D000014A0E866F0F0E876F000E06D0A1
:101330000001510E866F0F0E876F000E886FA8ECAC
:1013400003F08CAE07D000014A0E866F0F0E876F38
:10135000000E06D00001510E866F0F0E876F000E33
:10136000886FA8EF03F0D9CFE6FFDACFE6FFFA0ED9
:10137000E3CFD9FFFB0EE3CFDAFFFD0EE35209E71F
:101380002D0EDE6EFC0EE31EE32AFD0ED8B4E3063E
:10139000E31EE652E652E652FD0EE124E76EFF0E32
:1013A000E220E46EE652F70EE3CFE6FFF70EE3CF5E
:1013B000E6FF23EC0AF0F90EE124E96EFF0EE220CD
:1013C000EA6E13EC0AF00AE110EC0AF009E113EC02
:1013D0000AF008E110EC0AF007E108D01EEC0AF070
:1013E00019EC0AF01EEC0AF019EC0AF01EEC0AF0F7
:1013F000DE6AF90EE126FF0EE222FF0EE3CFDAFFEE
:10140000E552FF0EE3CFD9FFE552FC0EE124E96E71
:10141000FF0EE220EA6EEECFF3FFEFCFF4FF1200F3
:10142000EF380F0B1200EF500F0B02E1EE52D88491
:101430001200EF380F0B300FDE6E1200EE500F0B64
:10144000300FDE6E1200FC0EE3CFE9FFFD0EE3CF9E
:10145000EAFF100EE66EEE6AEE6AEF6AD890FD0EB5
:10146000E336FE0EE336ED36ED36EF36FF0EE306DD
:1014700009E044EC0AF0EE5244EC0AF0EE5244EC7F
:101480000AF0EDD7E56E1200030EEF24E8B6EF6E1A
:10149000300EEF24E8BEEF6E000C0001AE6BAF6BB8
:1014A0008B868B8894869488C78E280EC66EB0C0B3
:1014B000C8FF9E9612009EA664D09E960001AEA321
:1014C00010D0AEB95ED0AFA139D0AFA33CD0AFB58C
:1014D00003D0C5AC12D015D0AFBB27D0C5AC4AD015
:1014E00019D0AEA525D0AEB94CD0AFA127D0AFA3AF
:1014F0002AD0AFB508D0C5BC04D0ACC0C9FFAF85F9
:101500001200AF932CD0AFB708D0C5BC03D0ADC08C
:10151000C9FF22D0AF93AF9522D0AFBB06D0C5ACE8
:1015200029D0AF93AF95AF971AD0AE89AE91120084
:10153000AEA727D0AEB925D0AFB103D0C580AF815B
:101540001200AFB304D0ABC0C9FFAF831200AFB776
:1015500008D0C5BC03D0C586AF871200AF93C58243
:101560001200AFB905D0C596C58AC588AF891200EB
:10157000AFBB03D0C584AF8B1200C9CFADF0AE892D
:10158000AE911200FE0E0001B115AB6FB2C0ACF00F
:10159000AF6BAE6BAE81AE839E861200FE0E000175
:1015A000B315AB6FB4C0ACF0B5C0ADF0AF6BAE6B04
:1015B000AE81AE859E861200010E0001B611AB6FA2
:1015C000AF6BAE6BAE81AE879E86120081B003D04A
:1015D000FC6A02EF00F0A3EC08F05CEC0DF00001F7
:1015E000140E836FCEEC02F0B7EC0BF017EC09F0A1
:1015F0001AEC09F089EC05F057EC0CF000013F0EF5
:10160000B06F4DEC0AF004EC01F0E1EC02F05BECA1
:101610000AF063EC0DF0000906E098EC05F077ECB9
:101620000CF012EC01F027EC04F00001C16F000196
:10163000C151620A31E05A0A2BE00F0A25E0010A83
:101640001FE0030A19E0010A13E0070A0DE0010A8E
:1016500007E0030A01E023D08C701AEC09F01FD0D8
:101660008C721AEC09F01BD08C741AEC09F017D0AC
:101670008C761AEC09F013D08C781AEC09F00FD0A4
:101680008C7A1AEC09F00BD08C7C1AEC09F007D09C
:101690008C7E1AEC09F003D051EC0BF000D0B5D7DA
:1016A00012000001CA0E866F0D0E876F000E886F44
:1016B000A8EC03F00001CE0E866F0D0E876F000EB2
:1016C000886FA8EC03F00001CA0E866F0D0E876FBD
:1016D000000E886FA8EC03F00001D50E866F0D0E8A
:1016E000876F000E886FA8EC03F00001B60E866FBE
:1016F0000F0E876F000E886FA8EC03F00001F70E45
:10170000866F0F0E876F000E886FA8EC03F0000144
:101710004C0E866F100E876F000E886FA8EC03F0DA
:10172000E1EC02F05BEC0AF027EC04F00001C46F7E
:101730000001C45109E0790A03E0200A01E005D064
:10174000FC6A02EF00F011D010D0B7EC0BF089EC7E
:1017500005F098EC05F057EC0CF01AEC09F004ECED
:1017600001F012EC01F002D000D0DAD71200000133
:10177000CA0E866F0D0E876F000E886FA8EC03F0FF
:101780000001CE0E866F0D0E876F000E886FA8ECDD
:1017900003F00001CA0E866F0D0E876F000E886F72
:1017A000A8EC03F00001D50E866F0D0E876F000EBA
:1017B000886FA8EC03F00001400E866F0E0E876F55
:1017C000000E886FA8EC03F00001CC0E866F0E0EA1
:1017D000876F000E886FA8EC03F00001010E866F82
:1017E0000F0E876F000E886FA8EC03F00001580EF3
:1017F000866F0F0E876F000E886FA8EC03F0000154
:10180000900E866F0F0E876F000E886FA8EF03F0A3
:10181000060EF66E020EF76E000EF86E000109005D
:10182000F550BC6F0900F550BD6F03E1BC6701D0F6
:101830003DD00900F550B76F0900F550B86F0900A9
:10184000F550B96F09000900F550E96E0900F5502F
:10185000EA6E090009000900F550BA6F0900F55059
:10186000BB6F09000900F6CFBEF0F7CFBFF0F8CF8D
:10187000C0F0B7C0F6FFB8C0F7FFB9C0F8FF00016D
:10188000BA5302E1BB5307E00900F550EE6EBA0708
:10189000F8E2BB07F9D7BEC0F6FFBFC0F7FFC0C074
:1018A000F8FF0001BC07000EBD5BBFD712000001AE
:1018B0006D0E866F0F0E876F000E886FA8EC03F019
:1018C00081A007D00001830E866F0F0E876F000E78
:1018D00006D00001760E866F0F0E876F000E886FA0
:1018E000A8EC03F08150010B0001C36F120081A02E
:1018F00013D00001C35125E100016D0E866F0F0E5C
:10190000876F000E886FA8EC03F00001830E866FCE
:101910000F0E876F000E12D00001C35112E00001BC
:101920006D0E866F0F0E876F000E886FA8EC03F0A8
:101930000001760E866F0F0E876F000E886FA8EC81
:1019400003F08150010B0001C36F1200226A20AE28
:10195000AFEF0CF01F6C201EE86A2022221E1BAE87
:10196000B7EF0CF01A6C1B1EE86A1B22221E46EC15
:101970000DF01BBEC7EF0CF022AE000C1A6C1B1E44
:10198000E86A1B22166C171EE86A1722000C22BE9A
:10199000BEEF0CF02388FF0C1AC026F01A501F026D
:1019A000F4CF19F0F3CF18F01B502002F4CF1BF046
:1019B000F3CF1AF01F02F3501926F4501A22E86AE6
:1019C0001B2226502002F3501926F4501A22E86AEE
:1019D0001B22000C18501D02F3CF14F0F4CF15F0A9
:1019E0001E02F3501526000EF420166E18501F022A
:1019F000F3501626000EF420176E18502002F350F4
:101A0000172619501D02F3501526F4501622000E09
:101A1000172219501E02F3501626F450172219509F
:101A20001F02F35017261A501D02F3501626F450C9
:101A300017221A501E02F35017261B501D02F35096
:101A400017261200176A166A156A146A200EE76EC6
:101A5000D890183619361A361B36143615361636FF
:101A600017361D50145C1E5015581F501658205024
:101A7000175809E31D50145E1E50155A1F50165A70
:101A80002050175A182AE72EE4D71200176A166A50
:101A9000100EE76ED8901A361B36163617361F50C2
:101AA000165C2050175805E31F50165E2050175A39
:101AB0001A2AE72EF0D71200470ED56E660ED66EA4
:101AC000D58EF2941200F2A407D00001670EC26F07
:101AD000E850D626F294010C000C1DEE00F02DEE1D
:101AE00000F0F86A239C08EC0CF0E6EC0AF0FDD755
:101AF0001200FFFFFFFFFFFFFFFFFFFFFFFFFFFFE2
:101B0000FFFFFFFFFFFFFFFFFFFFFFFFFFFFFFFFE5
:101B1000FFFFFFFFFFFFFFFFFFFFFFFFFFFFFFFFD5
:101B2000FFFFFFFFFFFFFFFFFFFFFFFFFFFFFFFFC5
:101B3000FFFFFFFFFFFFFFFFFFFFFFFFFFFFFFFFB5
:00000001FF
